:100000000C9434000C943E050C9464050C9451003F
:100010000C9480050C9451000C9451000C945100E8
:100020000C9451000C9451000C9451000C9451000C
:100030000C9451000C947C040C9451000C945100CD
:100040000C94E4030C9451000C9451000C94510056
:100050000C9451000C9451000C9451000C945100DC
:100060000C9451000C94510011241FBECFEFD4E02A
:10007000DEBFCDBF12E0A0E0B1E0EAEDF1E202C0E8
:1000800005900D92A23FB107D9F714E0A2EFB2E0BC
:1000900001C01D92A432B107E1F70E94B3050C9490
:1000A000EB100C9400002B985F982C9A289AFFCFA5
:1000B000BF92CF92DF92EF92FF920F931F93DF9345
:1000C000CF9300D0CDB7DEB785E201C08F5FE82FB8
:1000D000F0E0E25CFC4F90819A30C1F78D5F90E0D8
:1000E000825C9C4FFC01329720812A3209F000C3C8
:1000F000FC0131972081233209F0FAC2DC01E8E1EA
:10010000F4E08D91819384E0E432F807D1F720E0A8
:1001100011E033E0F32E02E0222331F540E030E03D
:10012000832F90E0FC01E85EFB4F855F9D4F50817F
:10013000FC018081581711F44F5F01C036E0463052
:1001400079F480910B03882351F41092FB021092F2
:10015000FA02109200030093050300930B0320E1C1
:100160003F5F3630E8F2C0C2213031F540E030E088
:10017000832F90E0FC01E85EFB4F8E5E9D4F508127
:10018000FC018081581711F44F5F01C037E0473000
:1001900079F480910B03813051F41092FB0210929C
:1001A000FA021092000380930103F0920B0320E106
:1001B0003F5F3730E8F298C2223041F540E030E04E
:1001C000832F90E0FC01E85EFB4F865E9D4F5081DF
:1001D000FC018081581711F44F5F01C036E04630B2
:1001E00089F410920A031092080360910A0381E0D7
:1001F00090E03A8349830E94DD1010930E0320E1C2
:1002000049813A813F5F3630D8F26EC2233041F5E2
:1002100040E030E0832F90E0FC01E85EFB4F8F5D13
:100220009D4F5081FC018081581711F44F5F01C030
:1002300035E0453089F410920A0310930803609169
:100240000A0381E090E03A8349830E94DD10109315
:100250000E0320E149813A813F5F3530D8F244C234
:10026000243041F540E030E0832F90E0FC01E85E6F
:10027000FB4F895D9D4F5081FC018081581711F41F
:100280004F5F01C033E0433089F410930A031092AA
:10029000080360910A0381E090E03A8349830E9459
:1002A000DD1010930E0320E149813A813F5F333026
:1002B000D8F21AC22530D1F540E030E0832F90E02B
:1002C000FC01E85EFB4F855D9D4F5081FC01808104
:1002D000581711F44F5F01C035E0453019F56091B2
:1002E0001D0460933C0380911E0480933D0382E0D3
:1002F00090E03A8349830E94DD1083E090E06091B2
:100300003D030E94DD1000930A03109208036091E0
:100310000A0381E090E00E94DD1010930E0320E1BB
:1003200049813A813F5F353048F2DEC1263041F5E0
:1003300040E030E0832F90E0FC01E85EFB4F8F5CF3
:100340009D4F5081FC018081581711F44F5F01C00F
:1003500035E0453089F410920A0310920803609149
:100360000A0381E090E03A8349830E94DD101093F4
:100370000E0320E149813A813F5F3530D8F2B4C1A4
:10038000273009F056C030E040E0842F90E0FC01B7
:10039000E85EFB4F895C9D4F5081FC0180815817BE
:1003A00011F43F5F01C042E03230F1F58091170453
:1003B0008823C9F5809107038530A8F5809107034C
:1003C0008F5F809307038091070390E024E0880FFC
:1003D000991F2A95E1F7909316038093150388E1FE
:1003E000C82E84E0D82EF60181916F018093170307
:1003F0008091150390911603609117033A830E9430
:10040000DD108091150390911603019690931603C9
:10041000809315033A81F4E2CF16F4E0DF0619F772
:1004200000930E034CE020E14F5F423008F4ADCF63
:100430005BC12830F1F45091170440E030E0832F85
:1004400090E0FC01E85EFB4F865C9D4F6081FC0103
:100450008081681711F44F5F01C033E0433029F405
:10046000552311F400930E0320E13F5F333038F33E
:100470003BC1293031F540E030E0832F90E0FC01B2
:10048000E85EFB4F825C9D4F5081FC0180815817D4
:1004900011F44F5F01C036E0463079F410930F033A
:1004A00060910F0384E090E03A8349830E94DD105D
:1004B00010930E0320E149813A813F5F3630E8F224
:1004C00013C12A3031F540E030E0832F90E0FC0189
:1004D000E85EFB4F8B5B9D4F5081FC01808158177C
:1004E00011F44F5F01C037E0473079F410920F03E9
:1004F00060910F0384E090E03A8349830E94DD100D
:1005000010930E0320E149813A813F5F3730E8F2D2
:10051000EBC02B30B1F5C0901C04D0901D04E090CE
:100520001E04B0911F04A0911A0370911B036091E7
:100530001C0350911D0340E030E0832F90E0FC014C
:10054000E85EFB4F835B9D4FB080FC018081B81655
:1005500011F44F5F01C034E0443039F4F0920E03DF
:100560005B2F6E2D7D2DAC2D20E13F5F343028F3C5
:10057000A0931A0370931B0360931C0350931D03F5
:10058000B3C02C30D1F440E030E0832F90E0FC0188
:10059000E85EFB4F8E5A9D4F5081FC0180815817B9
:1005A00011F44F5F01C033E0433019F410930E0390
:1005B00020E13F5F333048F397C02D3031F540E004
:1005C00030E0832F90E0FC01E85EFB4F8A5A9D4F9C
:1005D0005081FC018081581711F44F5F01C036E053
:1005E000463079F4109310036091100385E090E099
:1005F0003A8349830E94DD1010930E0320E1498164
:100600003A813F5F3630E8F26FC02E3031F540E07E
:1006100030E0832F90E0FC01E85EFB4F835A9D4F52
:100620005081FC018081581711F44F5F01C037E001
:10063000473079F4109210036091100385E090E048
:100640003A8349830E94DD1010930E0320E1498113
:100650003A813F5F3730E8F247C0EE2430E02FE0C8
:10066000832F90E0FC01E85EFB4F8B599D4F40814A
:10067000FC018081481711F4E39401C034E0FE2DA1
:10068000F43071F580911704882349F5CC24DD24DA
:10069000C60140966FEF0E94DD100894C11CD11C6A
:1006A00080E5C816D104A1F71092100360911003E1
:1006B00085E090E00E94DD1010920F0360910F031F
:1006C00084E090E00E94DD1010920A03109208036B
:1006D00060910A0381E090E00E94DD1030E620E1A5
:1006E0003F5F343008F4BCCF2F5F203108F414CDC5
:1006F0000F900F90CF91DF911F910F91FF90EF908E
:10070000DF90CF90BF90089520E01092F3021092F6
:10071000F20207C08091F2029091F30284369105B3
:1007200028F48091C00087FFF5CF01C024E68091B6
:10073000C600E22FF0E0E25CFC4F80832F5F24369E
:1007400020F302C08091C6008091C00087FDFACFDF
:10075000089520E01092F3021092F20207C08091F7
:10076000F2029091F3028436910528F48091C00042
:1007700087FFF5CF01C02EE1E22FF0E08091C600A7
:10078000E25EFC4F80832F5F2E3120F302C0809108
:10079000C6008091C00087FDFACF08951F93CF93C4
:1007A000DF9310E0C12FD0E00E946A0FC25EDC4FE1
:1007B00088838881882309F41EE11F5F1E3190F32E
:1007C000DF91CF911F9108951F920F920FB60F9254
:1007D00011242F938F939F938091F6029091F702AB
:1007E00001969093F7028093F6028091F202909125
:1007F000F30201969093F3028093F2028091F40247
:100800009091F50201969093F5028093F402809105
:10081000F6029091F70227E180379207C0F010921C
:10082000F7021092F6028091FD028F5F8093FD0225
:1008300081E0809309039091FD029A3040F010927C
:10084000FD0290910603992311F480930603809191
:10085000F4029091F50228E08E35920708F444C026
:100860001092F5021092F40280910203813039F463
:100870008091FC02882311F42B9801C02B9A80915F
:100880000303813039F48091FC02882311F42C9801
:1008900001C02C9A80910403813039F48091FC02CC
:1008A000882311F45F9801C05F9A8091050381301D
:1008B00029F48091FC02882349F40AC08091050341
:1008C000823039F48091FC02882311F4289A01C007
:1008D00028988091FC028F5F8093FC028091FC023B
:1008E000823010F01092FC029F918F912F910F9007
:1008F0000FBE0F901F9018951F920F920FB60F9278
:1009000011248F939F9380910B03833009F042C091
:100910008091FA029091FB0201969093FB028093E2
:10092000FA028091FA029091FB028038910528F139
:100930001092FB021092FA02809100038F5F809365
:100940000003809100038D32C0F081E080930C039E
:100950004B9B07C010920B0310920503289884E06C
:100960000AC04B990AC080930B03809305038091C2
:100970000F03813011F480930E03809101038130C5
:1009800009F03FC01092010310920B03109205036F
:10099000289831C080910B03823099F58091FA023A
:1009A0009091FB0201969093FB028093FA02809152
:1009B000FA029091FB028038910518F11092FB0227
:1009C0001092FA02809100038F5F80930003809160
:1009D00000038D32B0F04B9B07C010920B031092B6
:1009E0000503289884E00BC04B990BC081E08093ED
:1009F0000B038093050380910F03813011F48093E2
:100A00000E0380910A03813039F58091080381300B
:100A100019F55E9A8091F8029091F90201969093EF
:100A2000F9028093F8028091F8029091F9028436DD
:100A30009105E8F01092F9021092F8028091FF02FD
:100A40008F5F8093FF028091FF02853080F01092CB
:100A5000FF02109208030AC080910A03882339F428
:100A600080910803813011F45E9A01C05E989F91D5
:100A70008F910F900FBE0F901F9018951F920F929D
:100A80000FB60F9211248F934A9908C01092030356
:100A90002C98419A81E08093020309C04A9B07C0C9
:100AA000419881E080930303109202032B98809178
:100AB0001003813019F482E0809306038F910F9028
:100AC0000FBE0F901F9018951F920F920FB60F92A6
:100AD00011248F9380910B03813061F482E0809325
:100AE00005031092FB021092FA021092000383E0B9
:100AF00080930B038F910F900FBE0F901F9018954E
:100B00001F920F920FB60F9211248F93329925C026
:100B100080910B03833021F481E0809301031DC099
:100B200080910B03882351F41092FB021092FA0279
:100B30001092000382E0809305030DC080910B03A7
:100B4000813059F41092FB021092FA0210920003C5
:100B50008093010383E080930B038F910F900FBE6E
:100B60000F901F9018953F924F925F926F927F92D5
:100B70008F929F92AF92BF92CF92DF92EF92FF92AD
:100B80000F931F93CF93DF9315B889E184B904E0E5
:100B900008B983E187B988E08BB982ED8AB98FEF14
:100BA00080BF80916E00816080936E0012E015BD61
:100BB00080916F00816080936F0081E0809381005D
:100BC00083E390E00E94480F8DE08093690083E00A
:100BD0008DBB00936C001093680080E88FBF84E0A9
:100BE0000E94630E8FEF99E6A8E181509040A040EB
:100BF000E1F700C000001092FE0215E026C08091CF
:100C0000FE0290E0019654E0880F991F5A95E1F793
:100C1000909316038093150380911503909116030A
:100C20000E94D51080931703809117038F3F31F0F6
:100C3000809107038F5F8093070302C01093FE0229
:100C40008091FE028F5F8093FE028091FE028530CC
:100C5000B0F281E090E00E94D51080930A03AFE1EA
:100C6000BEE41197F1F700C0000082E090E00E941E
:100C7000D51080933C038FE19EE40197F1F700C00B
:100C8000000083E090E00E94D51080933D03AFE127
:100C9000BEE41197F1F700C0000084E090E00E94EC
:100CA000D51080930F038FE19EE40197F1F700C008
:100CB000000085E090E00E94D51080931003AFE122
:100CC000BEE41197F1F700C00000409A8FE19EE466
:100CD0000197F1F700C00000449A5F9A359BFECF60
:100CE00044988FEF99E6A8E181509040A040E1F749
:100CF00000C000000E94940F882311F40E9453004A
:100D000080E091E060E20E945A0F0E94EF0F88237A
:100D100059F480E091E060E20E945A0F0E94EF0FC8
:100D2000882311F40E94530081E291E06EE10E9459
:100D30005A0F0E94EF0F882311F40E94530080E4A1
:100D400091E064E10E945A0F0E94EF0F882311F492
:100D50000E9453001092FE0211E036C08FEF99E618
:100D6000A8E181509040A040E1F700C000000E943F
:100D70007C0F85E591E06AE00E945A0F0E94840F83
:100D8000882311F10E94CE03809123038534D1F48E
:100D9000809124038734B1F480912903813369F071
:100DA000823318F4803371F405C0833319F085332E
:100DB00049F403C00E94530007C01093040310932A
:100DC000FE0202C01092FE028091FE02882331F2E0
:100DD0004A9905C0419A81E08093020305C04A9B6D
:100DE00003C081E080930303109206038091070300
:100DF000882359F082E08093050380930B031092BF
:100E0000FB021092FA021092000340E2E42E30E25C
:100E1000F32E25E0B22E9EE0A92E8DE0682E05E28D
:100E2000502E1EE1412EBEE13B2E80910C038130FD
:100E300009F09FC010920C031092FE0238C08091FE
:100E4000FE0290E00196A4E0880F991FAA95E1F7B1
:100E500090931603809315031092B20317C08091EC
:100E60001503909116030E94D510E12FF0E0EC5588
:100E7000FC4F808380911503909116030196909307
:100E80001603809315031F5F1093B2031091B203F2
:100E90001C3028F380E691E060E144EA53E02CE066
:100EA0000E948B108091FE028F5F8093FE029091D2
:100EB000FE0280910703981710F282E190E0909370
:100EC00016038093150388E38093A40381E0809345
:100ED000B20317C080911503909116030E94D5109C
:100EE000E12FF0E0EC55FC4F808380911503909149
:100EF0001603019690931603809315031F5F1093BA
:100F0000B2031091B2031B3028F31092FE0224C0EA
:100F10008FEF93EDA0E381509040A040E1F700C037
:100F2000000081E791E063E00E945A0F84EA93E0B9
:100F30006BE00E945A0F85E791E063E00E945A0F30
:100F40000E94EF0F813019F483E08093FE028091BC
:100F5000FE028F5F8093FE028091FE028330C0F21A
:100F60008FEF91E1AAE781509040A040E1F700C0E7
:100F7000000080910E03882309F495C280910E032E
:100F8000813011F01092110380911103882319F41C
:100F900081E0809311038091110390E0F4E0880FC9
:100FA000991FFA95E1F79093160380931503109219
:100FB000B20317C080911503909116030E94D510BB
:100FC000E12FF0E0EC55FC4F808380911503909168
:100FD0001603019690931603809315031F5F1093D9
:100FE000B2031091B2031C3028F380910E038130BC
:100FF00009F00CC180910B03882329F48FE48093BE
:10100000730286E416C080910B03813039F4F092AC
:1010100073028FE4809374028EE40DC080910B0301
:10102000823021F080910B03833039F48DE280937C
:1010300073028093740280937502809107028093FB
:101040007D028091080280937E0280910902809344
:101050007F0280910A028093810280910502809331
:101060008A028091060280938B0280911003813066
:1010700039F4F09292028FE4809393028EE40AC0D6
:1010800080911003882341F48FE48093920286E4D8
:1010900080939302809394024A9907C0F092990238
:1010A0008FE480939A028EE408C04A9B08C08FE4C4
:1010B0008093990286E480939A0280939B028091A8
:1010C000D8028093A9028091D9028093AA028091CC
:1010D0000803813039F4F092B1028FE48093B202B8
:1010E0008EE40AC080910803882341F48FE4809342
:1010F000B10286E48093B2028093B30280910A0326
:101100008823A9F484E78093B50282E78093B6022E
:1011100089E68093B70287E68093B802F092B9021D
:10112000F092BA02F092BB02F092BC021BC0809116
:101130000A038130F1F484E78093B50289E6809355
:10114000B6028DE68093B702F092B80285E38093F1
:10115000B90283E78093BA0285E68093BB0283E6F7
:101160008093BC02F092BD02F092BE02F092BF02E8
:1011700026C080910A03823011F584E78093B5027E
:1011800085E68093B6028DE68093B70280E7809370
:10119000B802F092B9028BE28093BA0280913C03CC
:1011A0008093BB0280913D038093BC028CE28093CC
:1011B000BD0280E38093BE0283E48093BF028091EE
:1011C0000F03813039F4F092CA028FE48093CB028E
:1011D0008EE40AC080910F03882341F48FE480934A
:1011E000CA0286E48093CB028093CC028AE692E026
:1011F00065E644EA53E02CE00E948B10813009F050
:1012000038C110920E03109211037FC080910E031B
:10121000823009F07DC01092FE020BC0E091FE0208
:10122000F0E0ED54FC4FE0828091FE028F5F8093EE
:10123000FE028091FE02843688F38091070380933A
:1012400017048DE48093B30381E48093B40383E5B2
:101250008093B50384E58093B60385E48093B70358
:1012600082E58093B803EAE07E2E3DC0C92DD0E030
:10127000CE0174E0880F991F7A95E1F790931603D9
:10128000809315032197CA9D802D11248A5F809336
:10129000A2031092B203C82FD0E08E010D541C4F50
:1012A00016C080911503909116030E94D510F80185
:1012B000E80DF11D8083809115039091160301962E
:1012C000909316038093150383948092B2038090C9
:1012D000B203B82DBC3028F3CD54DC4F6C867D862C
:1012E0009A949092170490901704992009F0BECF19
:1012F00083EB93E064E644EA53E02CE00E948B1019
:10130000813009F0B6C010920E0310921203B6C0DD
:1013100080910E03833009F0A4C08FEF99E6A8E115
:1013200081509040A040E1F700C0000004C08091CF
:10133000C6008093FE028091C00087FDF8CF89E748
:1013400091E064E00E945A0F8AE193E064E00E9419
:101350005A0F8EE791E062E00E945A0F1092FE024F
:101360007AC00E947C0F0E94840F8091C00087FF8A
:101370006DC00E94840380914203853509F066C0E8
:1013800080914303833509F061C080E08F5FE82FCF
:10139000F0E0E25CFC4F90819232C1F7282F8F5F22
:1013A000E82FF0E0E25CFC4F90819232C1F710929E
:1013B000FE020BC0E091FE02F0E0ED54FC4FE08233
:1013C0009091FE029F5F9093FE029091FE029436F0
:1013D00088F3922F9F5F9093FE0290E011C0A0913E
:1013E000FE02E92FF0E0ED54FC4FB0E0A25CBC4FF0
:1013F0002C9120839F5F2091FE022F5F2093FE029D
:101400002091FE02281758F39093FE028FEF9DE380
:10141000A9E481509040A040E1F700C00000609135
:10142000FE0283EB93E044EA53E02CE00E948B1031
:10143000813039F410920E03B092FE021092120322
:1014400005C0809112038F5F809312038091FE028A
:101450008F5F8093FE028091FE02853008F481CF79
:101460000DC080910E03843049F481E891E06BE176
:1014700042CF809112038F5F809312030E947C0FF2
:101480008DE991E065E10E945A0F0E94EF0F8130D3
:1014900019F41092120305C0809112038F5F80939C
:1014A00012030E947C0F80910903813009F0A7C1CB
:1014B0001092090380910A03813029F0809107037B
:1014C000882309F002C10E947C0F83EB91E069E060
:1014D0000E945A0F0E94840F8091C00087FFF5C0C0
:1014E0000E94A90380912303813409F0EEC080910A
:1014F0002403833509F0E9C080912703833309F081
:10150000E4C00E947C0F1092F3021092F20208C015
:101510008091F2029091F302AAE388399A0720F4AD
:101520008091C00087FFF4CF8091C00087FFCDC0BD
:101530001092B2031FC01092F3021092F2020AC07E
:101540008091F2029091F3028436910518F0409256
:10155000B20304C08091C00087FFF2CF8091B20334
:10156000E82FF0E09091C600E25EFC4F90838F5F21
:101570008093B2038091B2038E31E8F20E947C0F17
:10158000809122038E3409F0A0C080912303873418
:1015900009F09BC080912B03893409F096C080919B
:1015A0003103873309F091C080910703882379F5CF
:1015B00080E190E0909316038093150382E11AC0B6
:1015C000F0E0E25EFC4F8081809317038091150369
:1015D00090911603609117030E94DD10809115030E
:1015E00090911603019690931603809315038091B2
:1015F00017048F5F80931704E0911704EE3100F316
:1016000081E08093070382E080930E0359C08091AC
:101610000703882309F454C08091070380931704BB
:1016200062E1962E11E047C0802F90E054E0880FD1
:10163000991F5A95E1F79093160380931503109222
:10164000A3039092A20327C08091150390911603E3
:101650000E94D5108093170390911703E82DF0E0B6
:10166000E25EFC4F8081981731F48091A3038F5F75
:101670008093A30302C03092A2038091150390913E
:101680001603019690931603809315038091A2038D
:101690008F5F8093A2038090A203B82DBE31A0F289
:1016A0000150009317048091A3038C3021F4109310
:1016B00008031092170400911704002309F0B4CF17
:1016C0008DEB91E066E00E945A0F0E947C0F84EC43
:1016D00091E068E10E945A0F0E94840F8091C0003F
:1016E00087FF8DC00E948403809142038D3409F0EE
:1016F00086C0809144038C3409F081C08091070337
:10170000882309F462C0809107038093170409E1DC
:1017100057C0892D90E044E0880F991F4A95E1F762
:1017200090931603809315031092A3030093A203D2
:1017300027C080911503909116030E94D5108093C5
:10174000170390911703E12FF0E0E25CFC4F8081DA
:10175000981731F48091A3038F5F8093A30302C095
:101760005092A203809115039091160301969093D5
:101770001603809315038091A2038F5F8093A203C9
:101780001091A2031532A8F29A94909217048091B6
:10179000A3038C30A9F40E945800809117048F5F36
:1017A0008093110380E006C0E82FF0E0E25CFC4F7C
:1017B00010828F5F8E31C0F38093A20310921704C2
:1017C00090901704992009F0A4CF0E947C0F8DED12
:1017D00091E065E10E945A0F1092F3021092F2021A
:1017E00008C08091F2029091F30224E08C349207B9
:1017F00020F48091C00087FFF4CF0E947C0F80917D
:101800000603882309F411CB80910603823019F472
:1018100081E080930E03109206031092F30210925F
:10182000F2028091F2029091F30233E0803293074A
:10183000C0F30E947C0F83EF91E068E00E945A0F92
:101840000E94840F8091C00087FF30C00E94A903CE
:1018500080912203823451F580912303833431F542
:1018600080912B038C3229F48AE58093050282E56E
:101870000AC080912B038C3241F080912803809321
:10188000050280912903809306028091260380330C
:1018900031F44A990BC0109202032B9A07C0809131
:1018A0002603813319F481E0809302031092F3023E
:1018B0001092F2028091F2029091F302A3E0803242
:1018C0009A07C0F30E947C0F8CEF91E068E00E94C1
:1018D0005A0F0E94840F8091C00087FF12C00E949F
:1018E000A90380912203833561F48091230381351C
:1018F00041F4809126038093D8028091270380933E
:10190000D90284E00E94C30E84E00E94510D84E459
:1019100064E00E94270D84E00E94A30E8823D9F37F
:1019200084E00E94C30E84E00E94510D8EEB64E0BF
:101930000E94270D84E00E943E0D8093180384E0EE
:101940000E943E0D809319038091190387FD04C006
:101950008BE28093070213C08DE28093070290917F
:10196000190380911803D92ECC2490E08C299D294D
:10197000909581959F4F80931803909319039091B0
:1019800019038091180382958F709295907F890F2B
:101990008093140390910A039230A9F490913D032F
:1019A000905120913C03220F322F330F330F320F0F
:1019B000930F891728F481E0809308035E9A03C08F
:1019C0005E981092080320911403822F6AE00E940F
:1019D000C910805D8093080290910802205F86EF15
:1019E000989F802D1124280F2093090280911803BD
:1019F0008F70809314038A3060F48830E0F4843070
:101A0000A1F0853018F4823060F00DC0873078F096
:101A100010C08C30A1F08C3080F08F3090F08F307F
:101A200091F080E311C081E30FC082E30DC083E336
:101A30000BC084E309C085E307C086E305C087E3E4
:101A400003C088E301C089E380930A02EEC9FF92D4
:101A50000F931F93182FF62E08E010FF04C08F2D50
:101A60000E94710E03C08F2D0E948A0E015011F04A
:101A70001695F3CF1F910F91FF900895FF920F934A
:101A80001F93F82E08E010E016958F2D0E94A30EEC
:101A9000811110680150C1F7812F1F910F91FF90A4
:101AA0000895682F8CEC0E94270D08950F931F93C3
:101AB000CF93DF93EC01162F83E30E94270D08E0FC
:101AC000812F0E943E0D89930150D1F7DF91CF9174
:101AD0001F910F9108950F931F93CF93DF93EC0104
:101AE000062F85E50E94270D18E08991602F0E943E
:101AF000270D1150D1F7DF91CF911F910F910895CC
:101B0000CF92DF92EF92FF920F931F93CF93DF93C9
:101B1000EC01162F042F80EF642F0E94270DFF2465
:101B2000F394DD24EE24E394802F0E94A30EC82EAC
:101B3000802F0E94A30ECC2019F0882359F02CC0CE
:101B4000882331F09F2D909588818923888310C048
:101B5000E11619F488818F29F9CF98811E1528F490
:101B60008F2D80958923888302C09F2109F4DE2C64
:101B700088818F2121F0802F0E94710E03C0802F59
:101B80000E948A0EE394FF0C19F42196FF24F3942B
:101B90008E2D813449F602C0DD24DA948D2DDF913B
:101BA000CF911F910F91FF90EF90DF90CF9008950C
:101BB0006F927F928F929F92AF92BF92CF92DF925D
:101BC000EF92FF920F931F93DF93CF930F92CDB7B6
:101BD000DEB73C01D42E79018C01FC0180E0861730
:101BE00058F4108211821282138214821582168296
:101BF00017828F5F3896F3CF5301562D472DCC2493
:101C000060E08A2D9B2DFC01CA01292F342FD901B8
:101C100088E00D9001928150E1F78D2D69830E943B
:101C2000C30E6981882359F1C5014D2D0E94800D95
:101C3000682FC394882369F02C2D30E083E0220FB5
:101C4000331F8A95E1F7260D371D5A2D4B2D59016B
:101C5000D8CF20E0DD2410C0C80129830E940E0FD8
:101C60002981882329F4F70180818F5F808301C057
:101C700021E0D394085F1F4FDC1470F301C02FEFF5
:101C8000822F0F90CF91DF911F910F91FF90EF90D6
:101C9000DF90CF90BF90AF909F908F907F906F908C
:101CA0000895982F2F3F11F0822F08C080E007C0C1
:101CB000FB012081291731F0685F7F4F8F5F841708
:101CC000B8F38FEF089594B18095982394B995B1A6
:101CD000982395B98BEB93E00197F1F700C00000D2
:101CE00008952FB7F89494B1982B94B995B1809535
:101CF000982395B99AE09A95F1F700C094B198238A
:101D000094B995B1982395B985EA8A95F1F70000C1
:101D10002FBF08952FB7F89494B1982B94B995B12B
:101D20008095982395B99AE99A95F1F700C094B1F6
:101D3000982394B995B1982395B985E18A95F1F7DF
:101D400000002FBF08953FB7F89494B1982B94B931
:101D500095B1282F2095922395B99AE09A95F1F79D
:101D600000C094B1922394B995B1922395B922E120
:101D70002A95F1F700C093B12DE82A95F1F70000FC
:101D80003FBF892308953FB7F89494B1982B94B935
:101D900095B1282F2095922395B9EBEBF3E031977D
:101DA000F1F700C0000094B1922394B995B1922349
:101DB00095B9F5EBFA95F1F7000093B1EFE2F3E096
:101DC0003197F1F700C000003FBF90958923089537
:101DD00098E028E1362F382730FD02C0669503C011
:101DE000622766956068915011F08695F3CF862F33
:101DF000089598E022E030E4482F462740FD03C0D4
:101E00007695679505C06227732776956795706804
:101E1000915011F08695F0CFCB010895FF920F936A
:101E20001F93CF93DF93EC018C0167E0F62E60E007
:101E3000F80181918F010E94E80E682FFA94C1F792
:101E400081E09F81691709F480E0DF91CF911F91B4
:101E50000F91FF900895FF920F931F93CF93DF93FD
:101E6000EC018C0178E0F72E60E0F80181918F01A0
:101E70000E94E80E682FFA94C1F781E098856917EF
:101E800009F480E0DF91CF911F910F91FF900895A9
:101E90009093C5008093C40088E18093C10086E0E0
:101EA0008093C20008959091C00095FFFCCF80936D
:101EB000C6000895282F392FF90180E008C09091BD
:101EC000C00095FFFCCF91919093C6008F5F86175D
:101ED000B0F3089580E49DE0A3E0B0E004C0019772
:101EE000A109B10939F02091C00027FFF8CF8091F6
:101EF000C600089580E0089502C08091C6008091D8
:101F0000C00087FDFACF08958FEF9FEFDC0104C07A
:101F10000197A109B10931F02091C00027FFF8CF46
:101F200081E0089580E008957F928F929F92AF9212
:101F3000BF92CF92DF92EF92FF920F931F93DF93A6
:101F4000CF93CDB7DEB728970FB6F894DEBF0FBE9C
:101F5000CDBF25E0722E6E010894C11CD11C99E002
:101F6000A92EB12CAC0EBD1E88E0882E912C8C0EB3
:101F70009D1E0E947C0F8FED92E064E070E00E9455
:101F80005A0F860176010E946A0FF70181937F0143
:101F9000EA15FB05C1F7F80181918F018F3419F41F
:101FA00080818B3439F008151905A9F77A9409F75F
:101FB00080E001C081E028960FB6F894DEBF0FBE26
:101FC000CDBFCF91DF911F910F91FF90EF90DF90E8
:101FD000CF90BF90AF909F908F907F9008954F9239
:101FE0005F926F927F928F929F92AF92BF92CF92A9
:101FF000DF92EF92FF920F931F93DF93CF93CDB7B2
:10200000DEB7E1970FB6F894DEBF0FBECDBF8E01ED
:10201000075F1F4F88E2D8011D928A95E9F70E9459
:10202000840F009709F45FC020E029AB0E946A0F7B
:1020300029A9F801E20FF11D8083882309F428E221
:102040002F5F283290F380E005E4702E12E5C12E58
:10205000BFE4BB2EAEE38A2EF0E29F2EEBE4AE2E61
:1020600079E0472E512C4C0E5D1EAE014F5F5F4F45
:10207000813029F0823059F0B982AA820AC079826F
:10208000CA82CB82BC82CD8265E0D62E04C0898212
:102090009A8232E0D32E6980F20120E030E0919103
:1020A0009615C9F491E08A01020F131F692F70E0A1
:1020B0007801E60EF71E640F751FD7011896EC9095
:1020C000DB016C91E61294E69F5F9D1578F39D15F8
:1020D00011F48F5F09C02F5F3F4F28323105F9F6A9
:1020E0008F5F833029F680E0E1960FB6F894DEBF6B
:1020F0000FBECDBFCF91DF911F910F91FF90EF9059
:10210000DF90CF90BF90AF909F908F907F906F9017
:102110005F904F900895DF92EF92FF920F931F937D
:10212000CF93DF938C01F62EEA01D22E83E0E82EC6
:102130000E947C0F84EE92E069E070E00E945A0FEA
:10214000CE016D2D70E00E945A0F8EEE92E063E09A
:1021500070E00E945A0F0E94EF0F833069F4C801AB
:102160006F2D70E00E945A0F8AE190E00E94530F99
:102170000E94EF0F813021F0EA94D1F680E001C097
:1021800081E0DF91CF911F910F91FF90EF90DF9051
:102190000895991B79E004C0991F961708F0961BC3
:1021A000881F7A95C9F780950895F999FECF92BD59
:1021B00081BDF89A992780B50895262FF999FECF09
:1021C0001FBA92BD81BD20BD0FB6F894FA9AF99A54
:0A21D0000FBE01960895F894FFCFAA
:1021DA0041542B4950523D393630303B2B49464306
:1021EA003D302C303B2B4943463D332C333B0D0AC3
:1021FA000041542B434D47463D313B2B434C4950FC
:10220A003D313B2B434E4D493D323B45300D0A0093
:10221A0041542B434D4744413D2244454C20414CB7
:10222A004C220D0A0041542B435245473F0D0A00E8
:10223A00536563757269747920545245564F474104
:10224A0000415444003B0D0A0041544423000D0A46
:10225A00005365637572697479204F46460D0A45C5
:10226A0052524F52204441544348494B0041542B47
:10227A00434D4744413D2244454C2053454E542248
:10228A000D0A0041542B435041530D0A0041544852
:10229A00300D0A0041542B434D474C3D22524543D1
:1022AA0020554E52454144222C300D0A0041542BF0
:1022BA00434D4744413D2244454C20524541442226
:1022CA000D0A0041542B4342430D0A0041542B434B
:1022DA0053510D0A0030302B303030736563766B02
:1022EA006C007365636F746B6C0074726F746B6CE3
:1022FA00007472766B6C0074696D0074656D702B76
:10230A0000746F746B6C002B370074656C00736D0E
:10231A0073766B6C00736D736F746B6C0062616CB7
:10232A002A0073737300626174766B6C0062617465
:10233A006F746B6C003030303000536563757269AE
:10234A007479203132330D0A54656D70202B313285
:10235A002C34430D0A42617474203132252072658F
:10236A00702E31323320496E203132330D0A5369CF
:10237A00676E616C2047534D2031320D0A47504F2A
:10238A00203132332074726967202B31322C344366
:10239A000D0A534D53207265702E313233000000FE
:1023AA000000000000000000303041540D0A0041D6
:1023BA00540D0A0041542B434D47533D2200220D30
:0223CA000A0007
:00000001FF
